:100000002828A301A200FF30A207031CA307031C9A
:1000100023280330A100DF300F200328A101E83E90
:10002000A000A109FC30031C1828A00703181528FC
:10003000A0070000A10F152820181E28A01C2228A8
:100040000000222808008313831203130000080015
:1000500007309900FA30A400240801208316051106
:100060008312051524080120831685108312851438
:1000700024080120831605108312051483168512A7
:0A008000831285164228630043280E
:02400E00C43FAD
:00000001FF
